:03000000020008F3
:0300610002000397
:0500030012006480FE04
:100064007A017B007C0C7D000ABA00010B1CBCFFEA
:10007400011DEC4D70F28A088B09900086C002C005
:10008400031200FCAC82AD83D003D0028A088B0932
:10009400900086C002C003C004C005120142AE82B3
:1000A400AF83D005D004D003D0028A088B098C8298
:1000B4008D83C004C005C006C007120125E58285F2
:1000C40083F0D007D006D005D0042EFAEF35F0FB2C
:1000D4008C808E808A80BA8617BB0014BE0411BF40
:1000E400000EBC0A0BBD000875A0AA75B0AA800654
:1000F40075A05575B00180FE7A10E4FBFCE58225FD
:10010400E0F582E58333F583EB33FBEC33FCEB95CD
:1001140008F5F0EC95094006FCABF0438201DADD0A
:0101240022B8
:06003700E478FFF6D8FD9D
:100015007900E94400601B7A00900193780075A08F
:1000250000E493F2A308B8000205A0D9F4DAF2754A
:02003500A0FF2A
:10012500E5828508F0A4C582C0F08509F0A4D0F069
:1001350025F0C5838508F0A42583F58322E50845C8
:100145000960467A01E50825E0F508E5093340121E
:10015500F509E5829508E583950940030A80E6C31C
:10016500E50913F509E50813F508C3E5829508F5D2
:10017500F0E58395094005F58385F082C3E509130C
:0A018500F509E50813F508DAE12298
:10003D007800E84400600A790075A000E4F309D85F
:10004D00FC7800E84400600C7900900000E4F0A317
:04005D00D8FCD9FAF8
:0D00080075810912018FE58260030200037B
:04018F007582002253
:00000001FF
